:100000000C94EC020C9430030C9430030C943003E9
:100010000C9430030C9430030C9430030C94300394
:100020000C9430030C9430030C94460F0C9418106D
:100030000C9430030C9430030C9430030C94300374
:100040000C9430030C94D2230C9430030C943003A2
:100050000C9430030C94651D0C9430030C94300305
:100060000C9430030C9430030C9430030C94300344
:100070000C9430030C9430030C9430030C94300334
:100080000C9430030C9430030C9430030C94300324
:100090000C9430030C9430030C9430030C94300314
:1000A0000C9430030C9430030C9430039405C80571
:1000B000ED052B069405D1050F063906FA06FA065A
:1000C000BD06C706D106E3068510A7109511A71037
:1000D0009511EC100F119511641177114614461407
:1000E00075147514AB14CB14FC15FC15D614FC1543
:1000F00086158615ED15FC15FC15F615931593154B
:1001000093159315931593159315931593159315AF
:10011000931593159315931593159315A515B2156E
:10012000B915C015CA15000000000000000000004D
:10013000000000000000000000000AC80BC80CC846
:100140000DC80EC80FC810C811C80D200C200B30E8
:100150000A30E00000001E00140004001D0000072B
:100160004E001F001A0016001B00000F4C0020005C
:10017000080007000600E2002A002100150009001F
:100180001900E3004B00220017000A0005000000E0
:100190004A0029002F0000002B0200004D002D0016
:1001A000300000002B000000500023001C000B005A
:1001B000110000004F00240018000D001000E7009F
:1001C000520025000C000E003600E6002C00260030
:1001D00012000F003700000F280027001300330023
:1001E000380000075100112010200F200E30E400CD
:1001F00000000100010001000100E00000003A00E1
:100200001E0220022202000751003B001F022102B1
:100210002302000F28003C002F0226022F00E200DC
:100220002C003D00300227023000E30052003E0067
:10023000240235003502000050002900360200007B
:100240002B0000004F002D00370200002B020000A1
:100250004A003F0031023800310000004D004000EC
:10026000240021001E0027784B00410025002200B9
:100270001F0037744C0042002600230020002E7F10
:100280002A004300380025022D002E774E00010081
:1002900001000100010028710000010001000100BF
:1002A0000100E000000044006600A6000000000716
:1002B000B50045001430F2001630F600000068006A
:1002C000F000F100F100F400B60069001530F30011
:1002D0001730F500B4006A00A900AA00A8000000C9
:1002E000B8002900F9000000FA000000B900000081
:1002F000F9000000FA000000AC006B00460053005B
:1003000000000000AB006C004A0050004D0049782E
:10031000A9006D005200510051004C74AE006E00F7
:100320004B004F004E00000FAD006F00B100B30056
:1003300000000007AA000100010001000100E40024
:10034000000001000100010001000100000029007F
:100350000100010001000100010001000100010095
:100360000100010001000100010001000100010085
:100370000100010001000100010001000100010075
:100380000100010001000000010001000100000067
:100390000100000001000100010000000100000058
:1003A0000100010001000100010000000100010046
:1003B0000100010001000100010001000100010035
:1003C0000100010001000100010001000100010025
:1003D00001002A00010001000100010001000100EC
:1003E00001000100E5000100000016034500720055
:1003F00067006F0044006F007800200045005A003D
:10040000000016034500720067006F0044006F0093
:100410007800200045005A00000004030904090286
:100420006D00040100A0FA090400000103010100AD
:10043000092111010001223F000705810308000A7C
:100440000904010001030102000921110100012238
:100450004D000705820308000A0904020001030099
:10046000000009211101000122360007058303085D
:10047000000A090403000103000000092111010022
:100480000122390007058403100001120110010048
:10049000000008EDFE07130100010200010501093B
:1004A00006A101050719E029E71500250195087542
:1004B000018102050819012905950575019102952B
:1004C000017503910105071900297715002501958C
:1004D0007875018102C005010980A101850216011C
:1004E0000026B7001A01002AB70075109501810097
:1004F000C0050C0901A1018503160100269C021A02
:1005000001002A9C02751095018100C005010902B5
:10051000A1010901A10005091901290515002501FD
:100520009505750181029501750381010501093069
:1005300009311581257F95027508810609381581D5
:10054000257F950175088106050C0A38021581255D
:100550007F950175088106C0C005010906A1010546
:100560000719E029E7150025019508750181029515
:100570000175088101050819012905950575019185
:10058000029501750391010507190029FF15002542
:10059000FF950675088100C0000000000000000003
:1005A000000000010204060A0F17202C3A4A5D7170
:1005B000879DB3C7DAE9F5FCFFFCF5E9DAC7B39D1F
:1005C00087715D4A3A2C20170F0A060402010000C9
:1005D000000000000000000011241FBECFEFDAE091
:1005E000DEBFCDBF04B603FE24C08091030290910C
:1005F0000402A0910502B09106028730904BA740FB
:10060000B04BB9F41092030210920402109205024A
:100610001092060214BE84B7877F84BF88E10FB6AC
:10062000F89480936000109260000FBEE0E0FFE35A
:10063000099511E0A0E0B1E0E2E3FBE402C005901F
:100640000D92A433B107D9F712E0A4E3B1E001C0E1
:100650001D92A330B107E1F70E948A0C0C949725F4
:100660000C9400001092B9008AE08093B8000895BD
:1006700094EA9093BC009091BC0097FFFCCF9091BE
:10068000B900987F983021F0903111F081E0089501
:100690008093BB0084E88093BC008091BC0087FFFE
:1006A000FCCF8091B900887F883111F0803471F7D8
:1006B00080E0089584E98093BC008091BC0084FDB3
:1006C000FCCF08958093BB0084E88093BC008091A8
:1006D000BC0087FFFCCF9091B900987F81E09832F1
:1006E00009F480E0089584E88093BC008091BC0008
:1006F00087FFFCCF8091BB0008958091010181119B
:1007000015C080E40E9438038093010181110CC060
:1007100082E10E94620380930101811105C08FEF85
:100720000E946203809301010E945A0384B1807F7A
:1007300084B985B1807F85B98AB1837F8AB98BB14D
:10074000837F8BB93E98469808950E943805809320
:1007500001010E947D0380B38C7080BB81B3836FE5
:1007600081BBA5E3B1E0E3E4F1E08EE08E0F1192EE
:100770001D928E13FCCF0C942205BF92CF92DF9274
:10078000EF92FF920F931F93CF93DF93809101011C
:10079000882379F0809134018F5F80933401811137
:1007A00008C00E94380580930101811102C00E9497
:1007B000CA0405E311E0C0E0D0E0DD24D39482E078
:1007C000C82EEE24E394F12CC730D10500F58091BA
:1007D0000101811164C080E40E943803809301010B
:1007E000811112C082E10E94620380930101811194
:1007F0000BC0C7010C2E01C0880F0A94EAF7809540
:100800000E946203809301010E945A0348C0CA30CB
:10081000A1F028F4C83059F0C93061F005C0CC30DF
:1008200089F070F0CD3089F0209A289810C0219A74
:1008300029980DC0229A2A980AC0239A2B9807C09B
:10084000529A01C0539A5B9802C03E9A469890EA29
:100850009A95F1F79FB1799902C082E001C080E0DA
:1008600091709D25982B7C9902C084E001C080E0A6
:10087000892B7D9902C038E001C030E0832B7E993E
:1008800002C020E101C020E0822B9FB19095991F0A
:100890009927991F9295990F907E892B0FC080916F
:1008A0000101811149C080E40E9438038093010155
:1008B000882379F1B12C0E945A038B2DF801908185
:1008C000981719F08083C09200010E947D03219641
:1008D0000F5F1F4FCE30D10509F076CF8091000118
:1008E000882361F1815080930001882339F08FE9DA
:1008F0009FE00197F1F700C0000020C0A3E4B1E041
:10090000E5E3F1E0CF01825F91919D938E13FCCFDF
:1009100015C083E10E946203809301018111CACF57
:1009200081E40E943803809301018111C3CF0E94AA
:100930007303B82EB094BFCF80E0C0CF0E94C8042C
:1009400081E0DF91CF911F910F91FF90EF90DF90A9
:10095000CF90BF900895E82FF0E0ED5BFE4F8081CF
:10096000089508950F931F93CF93DF93C3E4D1E0CD
:1009700010E00C2F025F899190E00E94DB1C180FA1
:100980000C13F9CF812FDF91CF911F910F91089513
:100990000C94FE0656985E9825982D9826982E98C9
:1009A00027982F988FEF90E090938900809388008C
:1009B00090938B0080938A0090938D0080938C009D
:1009C000259A2D9A2FEF80E792E0215080409040A9
:1009D000E1F700C00000269A2E9A2FEF80E792E000
:1009E000215080409040E1F700C00000279A2F9AE4
:1009F0002FEF80E792E0215080409040E1F700C067
:100A0000000025982D982FEF80E792E0215080403C
:100A10009040E1F700C0000026982E982FEF80E765
:100A200092E0215080409040E1F700C000002798FC
:100A30002F9856985E9825982D9826982E98279846
:100A40002F98089589EA8093800089E0809381003F
:100A500024982C983F988AB18F748AB96E98479AD7
:100A60008BB1806B8BB9769A0E94CA040C94FD06F8
:100A700080E2809301018091510181110EC00E949A
:100A8000320381E0809351012FEF83ED90E32150F9
:100A900080409040E1F700C0000080E40E943803ED
:100AA0008093010181112EC00E9462038093010195
:100AB000811128C00E94620380930101811122C02C
:100AC0008FE30E9462038093010181111BC00E9489
:100AD0005A0380E40E94380380930101811112C0FF
:100AE0008CE00E9462038093010181110BC00E947F
:100AF000620380930101811105C08FE30E946203AC
:100B0000809301010E945A03809101010895462FAC
:100B100050E0FA013A97EE30F10508F06BC1DC01C4
:100B2000EA5AFF4F0C94472512962C911297809108
:100B30005801909159012223F9F015962C91207FAC
:100B4000D9F401968330910510F082E090E0909303
:100B50005901809358018091580190915901823038
:100B6000910529F489E30E94EA1289E30EC00197F6
:100B700009F040C181EEFAC001979093590180932A
:100B80005801892B09F036C181EE0E94B21332C19F
:100B900012962C918091560190915701222379F061
:100BA00090C012963C91129715962C918091560107
:100BB00090915701207F31117AC009F09FC00197B1
:100BC0009093570180935601892B09F013C18091AE
:100BD000530181110FC181E067C012963C911297B9
:100BE00015962C918091540190915501207F3323CB
:100BF00061F0222309F491C0009709F08EC0209182
:100C0000520121118AC08BE2B1C02223B1F00097BA
:100C1000A1F420915201211110C08BE2B6CF12969F
:100C20003C91129715962C91809154019091550109
:100C3000207F311168C009F08DC001979093550154
:100C400080935401892B09F0D5C080915201811104
:100C5000D1C082E029C012969C91129715968C9172
:100C60009923B1F0982F907F79F080FD0DC085E336
:100C70007DC012969C91129715968C91992379F0CC
:100C8000982F907F09F06FC083E00E94A41AB2C031
:100C9000982F907F41F080FD06C085E376CF982F96
:100CA000907F09F066C083E00E94C51AA3C022238A
:100CB00041F0009731F420915301211102C084E3E7
:100CC00055C001968330910510F082E090E090933A
:100CD00057018093560180915601909157018230BF
:100CE000910529F0019709F085C081E0CECF909160
:100CF000530181E08927809353017CC0009709F05C
:100D00005ECF84E342CF222341F0009731F420915B
:100D10005201211102C081E329C00196833091055F
:100D200010F082E090E090935501809354018091FF
:100D30005401909155018230910529F0019709F0F5
:100D400059C082E0A2CF9091520181E0892780931F
:100D5000520150C0009709F070CF2091520121112B
:100D60006CCF81E312CF80FD8FCF8EE20E94EA121A
:100D700041C080FD98CF8EE208CF12968C918823D7
:100D800019F080EF90E013C080EF90E017C012964A
:100D90008C91882319F080EF90E01BC080EF90E0E9
:100DA00021C012968C91882339F081EF90E00E9447
:100DB000D71F82EF90E011C081EF90E00E943F20AA
:100DC00082EF90E013C012968C91882349F081EF56
:100DD00090E00E94D71F83EF90E00E94D71F08C0C9
:100DE00081EF90E00E943F2083EF90E00E943F203F
:100DF0000E94C42080E090E00895089580915801F9
:100E000090915901892B19F0259A2D9A0DC0E091E6
:100E10000E01F0910F01808185FDF6CF0E94CE1169
:100E200081FDF2CF25982D988091C50181FF03C0E7
:100E3000269A2E9A02C026982E988091C50182FF8C
:100E400003C0279A2F9A089527982F98089581E034
:100E5000089581E008950C94290708950F931F9336
:100E6000CF93DF938C01FC01C081D181CE010E9420
:100E7000601BBE010E94D707EC01B8010E942B073E
:100E8000882309F48DC0F8018281882309F44AC0BF
:100E90008091650181111FC0C431F0E5DF0709F0C1
:100EA00051C00E942D0781E0809365010E942F1D93
:100EB000909364018093630110925C0110925E0133
:100EC00010925D011092600110925F011092620118
:100ED0001092610165C080916301909164010E944C
:100EE0003B1D883C910570F480915C01E82FF0E097
:100EF000EE0FFF1FE35AFE4FD183C0838F5F8093B5
:100F00005C014EC0C43880E5D80721F0C538D04513
:100F100001F13AC0F8018281882341F010925A0110
:100F200082E01EC0C438E0E5DE0759F580915A0121
:100F3000811106C086E20E94EA1286E20E94B21384
:100F400082E01CC0C438F0E5DF0741F3C538D04566
:100F5000D9F4F8018281882331F010925B0180E29C
:100F60000E9401141DC080915B01811106C087E2BF
:100F70000E94EA1287E20E94B21380E20E940814E3
:100F80000FC0C538D04529F381E080935A01809382
:100F90005B01C801DF91CF911F910F910C9427073E
:100FA00080E0DF91CF911F910F910895089596E011
:100FB000799FF001112494E5899FE00DF11D112422
:100FC000E60FF11DEE0FFF1FE65BFE4F859194913A
:100FD0000895880F991FFC01EA55F040859194917E
:100FE0000895880F991FFC01EA5DFE4F8591949149
:100FF00008950F931F93CF93DF93EC01811520E3A6
:10100000920750F5C11580E2D80708F0C3C0CB3B6A
:10101000D10590F4C83AD10508F06AC0C53AD105A7
:1010200008F05BC0C430D10508F0D0C1219709F0A9
:10103000CAC101E010E00AC2CF3FD10511F008F0AB
:10104000C5C1C03FD10508F0A2C0CE01805E9109A4
:10105000089708F4BBC1B7C1C13090E5D90709F4BE
:10106000A2C020F5C0318FE4D80770F4C11590E418
:10107000D90708F094C0C11521E3D20708F0A3C135
:10108000DD278E01106CE2C1C115D04509F09BC16E
:101090000E9467168FEF94E32CE08150904020402F
:1010A000E1F700C000000E948A1DD0C1C11597E57C
:1010B000D90758F4C03121E5D20708F01CC1C4316A
:1010C00080E5D80708F475C07EC1CE019057811520
:1010D000904108F078C1DF7073C1C53AD10509F4B9
:1010E00077C1C63AD10509F076C102E810E4AEC175
:1010F000C83AD10509F472C1C93AD10509F471C1E0
:10110000CA3AD10509F470C1CB3AD10509F46FC1CF
:10111000CC3AD10509F46EC1CD3AD10509F46DC1BF
:10112000C03BD10509F46CC1CE3AD10509F46BC1BD
:10113000CF3AD10509F46AC1C13BD10509F469C1AF
:10114000C23BD10509F468C1C33BD10509F467C1AD
:10115000C43BD10509F466C1C53BD10509F465C19D
:10116000C63BD10509F464C1C73BD10509F463C18D
:10117000C83BD10509F462C1C93BD10509F461C17D
:10118000CA3BD10509F460C100E014E45FC18E01DF
:1011900010655CC1CE019F700E94F10758C1DF70DD
:1011A0008E01106A53C18091E20181608093E20157
:1011B0004DC10E942F1F811102C00E94151F0E9465
:1011C0004C1F90E09093030280930202C23080E5AE
:1011D000D80721F480910202816086C0C43090E576
:1011E000D90721F48091020282607EC0C63020E5DA
:1011F000D20721F480910202846076C0C83080E575
:10120000D80719F48091020227C0CA3090E5D907A7
:1012100021F480910202806167C0CC3020E5D207C2
:1012200021F48091020280625FC0CE3080E5D80751
:1012300021F480910202806457C0C03190E5D90743
:1012400021F48091020280684FC0C23120E5D207AC
:1012500029F4809102028460886046C0C33080E532
:10126000D80721F4809102028E7F3EC0C53090E500
:10127000D90721F4809102028D7F36C0C73020E566
:10128000D20721F4809102028B7F2EC0C93080E505
:10129000D80719F48091020226C0CB3090E5D90717
:1012A00021F4809102028F7E1FC0CD3020E5D2074D
:1012B00021F4809102028F7D17C0CF3080E5D807DE
:1012C00021F4809102028F7B0FC0C13190E5D907D4
:1012D00021F4809102028F7707C0C331D04531F4E9
:1012E000809102028B7F877F8093020280910202AD
:1012F0000E94501FABC08D2F99278F709927813086
:101300009105D9F49E012370332702C0880F991FDD
:101310002A95E2F79C688E0144E0000F111F4A9560
:10132000E1F700271370802B912B53E0CC0FDD1FCA
:101330005A95E1F7C076DD272FC08230910531F450
:10134000DC2FCC278E01016F106A80C0833091059D
:1013500069F4CE018370992701E010E002C0000F0C
:10136000111F8A95E2F7C8019C680FC0843091056F
:10137000B9F4CE018370992701E010E002C0000F9C
:10138000111F8A95E2F7C8019A6823E0CC0FDD1F90
:101390002A95E1F7C07ED7708C010C2B1D2B56C00F
:1013A0008530910531F4DC2FCC278E01046F106A53
:1013B0004DC0069709F04AC0CF71DD27DC2FCC273E
:1013C0008E01106243C000E010E040C08E013EC0BC
:1013D00001E810E43BC003E810E438C002EE14E476
:1013E00035C009EE14E432C00AEE14E42FC005EB58
:1013F00014E42CC006EB14E429C007EB14E426C067
:101400000CEC14E423C00DEC14E420C003E815E454
:101410001DC00AE815E41AC002E915E417C004E982
:1014200015E414C001E216E411C003E216E40EC094
:1014300004E216E40BC005E216E408C006E216E476
:1014400005C007E216E402C00AE216E4C801DF9113
:10145000CF911F910F91089596E0799FF00111248B
:1014600094E5899FE00DF11D1124E60FF11DEE0FAB
:10147000FF1FE65BFE4F85919491803E9105E0F45D
:10148000803C910558F58133910509F46FC048F40B
:101490008932910509F463C08A32910509F46DC05F
:1014A00072C089339105E9F082389105D1F0853316
:1014B000910509F44DC067C0833E910581F138F470
:1014C000803E9105B9F0823E9105D9F05CC0863E20
:1014D000910561F1873E9105A1F155C00E94E90790
:1014E00008952091020220FD02C021FF4CC080EE31
:1014F00090E049C08091020280FFF9CF89E390E03B
:1015000042C08091020282FF0EC08091020284FFDD
:1015100003C080E090E037C083EE90E034C080915B
:10152000020282FFF2CF82EE90E02DC08091020293
:1015300083FF0BC08091020284FDEBCF87EE90E029
:1015400022C08091020283FFF5CF86EE90E01BC09F
:101550008091020285FF07C089E290E014C080916B
:10156000020285FFF9CF85E390E00DC08091020271
:1015700086FF07C08AE290E006C08091020286FFE3
:10158000F9CF81E390E00E94F907089508950C9443
:10159000C60A809176010895CF93DF9300D01F9201
:1015A000CDB7DEB79C018091F901843019F593E045
:1015B00099833B832A839093E9008FEF9091E80011
:1015C000815095FD06C095ED9A95F1F700008111C7
:1015D000F5CF8091E80085FF0DC040E050E063E06A
:1015E00070E0CE0101960E94360D8091E8008E7762
:1015F0008093E8000F900F900F90DF91CF910895A6
:10160000CF93DF9300D01F92CDB7DEB72091F901C1
:10161000243021F522E029839B838A8383E0809311
:10162000E9008FEF9091E800815095FD06C095ED9F
:101630009A95F1F700008111F5CF8091E80085FFC0
:101640000DC040E050E063E070E0CE0101960E94E2
:10165000360D8091E8008E778093E8000F900F9010
:101660000F90DF91CF9108952091F9012430F1F48A
:1016700022E02093E9002FEF3091E800215035FD62
:1016800006C035ED3A95F1F700002111F5CF209114
:10169000E80025FF0BC040E050E065E070E00E94EC
:1016A000360D8091E8008E778093E8000895CF93FF
:1016B000DF93EC019091F901943009F046C08091DC
:1016C0000C018823D9F080910D018823B9F0909303
:1016D000E9008FEF9091E800815095FD06C095E1FB
:1016E0009A95F1F700008111F5CF8091E80085FF10
:1016F0002CC040E050E060E170E017C081E08093D2
:10170000E9008FEF9091E800815095FD06C095EDBE
:101710009A95F1F700008111F5CF8091E80085FFDF
:1017200014C040E050E068E070E0CE010E94360D49
:101730008091E8008E778093E80080E1FE01A6E6C4
:10174000B1E001900D928A95E1F7DF91CF91089574
:101750008091F801811109C00E94CB0E0E94280FD0
:101760008091E20084608093E20008951092F80175
:10177000089508950C94BF230E94201D0E94C52344
:101780000E94CE110C94C70A42E061EC81E00E94F5
:10179000450E42E061EC82E00E94450E42E061ECC1
:1017A00083E00E94450E42E161EC84E00C94450E1A
:1017B0008091FB01833009F455C030F4813071F021
:1017C000823009F48EC008958A3009F47AC08B30D3
:1017D00009F460C0893009F09CC020C08091FA01F2
:1017E000813A09F096C08091E800877F8093E800F5
:1017F0008091FE019091FF01892B21F460E186E642
:1018000091E003C060E080E090E070E00E94810D14
:101810008091E8008B778093E80008958091FA0129
:10182000813209F076C08091FE019091FF0100970E
:1018300019F0039709F06DC08091E800877F8093CD
:10184000E8008091E80082FD05C08091F9018111D6
:10185000F8CF5FC08091F100809376018091E8001D
:101860008B7753C08091FA01813A09F052C0809180
:10187000FE019091FF01892B09F04BC08091E80097
:10188000877F8093E8008091E80080FFFCCF809103
:101890000C0136C08091FA018132D9F58091FE01A8
:1018A0009091FF01892BA9F58091E800877F8093B3
:1018B000E8000E947A0E8091FC0180930C010C9448
:1018C00067168091FA01813221F58091E800877FC7
:1018D0008093E8000E947A0E8091FD018093770149
:1018E00008958091FA01813AA1F48091E800877F00
:1018F0008093E8008091E80080FFFCCF8091770121
:101900008093F1008091E8008E778093E8000C943A
:101910007A0E089584B7877F84BF88E10FB6F89464
:1019200080936000109260000FBE90E080E80FB6D8
:10193000F89480936100909361000FBE0E941D1285
:101940000E94CB0E0E94280F8091E2008460809359
:10195000E20078940E94AE110E941F1282E091E092
:101960000E94C9110E94AD238091F901853069F46C
:101970000E94E71C8091F7018823B1F30E94121D99
:10198000882391F30E94200DEFCF0E942512ECCF07
:10199000292F332723303105C9F064F42130310574
:1019A00081F02230310509F043C08DE690E02EE150
:1019B00034E042C021323105F1F02232310541F1EB
:1019C00037C082E190E02BE834E036C099278130BF
:1019D000910541F08230910541F0892B49F5EAE10A
:1019E000F4E005C0E2E0F4E002C0EAEEF3E0849146
:1019F00090E09F0121C06430D8F4E62FF0E0EE0FB4
:101A0000FF1FEE5DFE4F2081318189E090E014C020
:101A1000643070F470E0FB01EE0FFF1FE65EFE4FD6
:101A200020813181FB01EA5EFE4F808190E004C09D
:101A300080E090E020E030E0FA01318320830895D7
:101A400080E189BD82E189BD09B400FEFDCF8091AE
:101A5000D8008F7D8093D8008091E00082608093D1
:101A6000E0008091E00081FDFCCF0895CF92DF92ED
:101A7000EF92FF920F931F93CF93DF93EC018B01B3
:101A80006A010E94990E811133C0C114D10439F04A
:101A9000F60180819181081B190BC80FD91FE12C19
:101AA000F12C0115110519F18091E80085FD16C092
:101AB0008091E8008E778093E800C114D10449F04A
:101AC000F60180819181E80EF91EF182E08285E0C5
:101AD0000FC00E94990E882321F30AC08991809338
:101AE000F10001501109FFEFEF1AFF0ADACF80E091
:101AF000DF91CF911F910F91FF90EF90DF90CF90EA
:101B0000089520910002309101022617370748F00E
:101B10006115710539F42091E8002E772093E800D3
:101B200001C0B90140E061157105A9F12091F901E9
:101B3000222309F443C0253009F442C02091E80073
:101B400023FD40C02091E80022FD32C02091E80032
:101B500020FFE9CF4091F3002091F20030E0342BD8
:101B6000FC01CF016115710559F02830310540F4B1
:101B700081918093F100615071092F5F3F4FF1CF48
:101B800041E02830310509F040E02091E8002E774F
:101B90002093E800C8CF4111C9CF0AC08091F90154
:101BA000882361F0853061F08091E80083FD0AC0F0
:101BB0008091E80082FFF2CF80E0089582E00895EE
:101BC00083E0089581E008952091000230910102A0
:101BD0002617370748F06115710539F42091E800A0
:101BE0002E772093E80001C0B901FC0120E06115C7
:101BF000710591F18091F901882309F440C0853085
:101C000009F43FC08091E80083FD3DC08091E80069
:101C100082FD2FC08091E80080FFE9CF2091F30082
:101C20008091F20090E0922B6115710559F0883097
:101C3000910540F424912093F1003196615071098F
:101C40000196F2CF21E0089709F020E08091E800AA
:101C50008E778093E800CBCF2111CCCF0AC0809142
:101C6000F901882361F0853061F08091E80083FDFF
:101C70000AC08091E80082FFF2CF80E0089582E000
:101C8000089583E0089581E00895982F973058F5DE
:101C90009093E900981739F07091EC002091ED00D5
:101CA0005091F00003C0242F762F50E021FF19C07F
:101CB0003091EB003E7F3093EB003091ED003D7FA3
:101CC0003093ED003091EB0031603093EB00709376
:101CD000EC002093ED005093F0002091EE0027FFE0
:101CE00007C09F5FD3CF8F708093E90081E0089594
:101CF00080E008958091FA0187FF11C08091E8008B
:101D000082FD05C08091F9018111F8CF11C0809149
:101D1000E8008B770BC08091F901882349F080910E
:101D2000E80080FFF8CF8091E8008E778093E8008C
:101D300008952091E4003091E50095E64091EC0093
:101D4000842F817040FF22C08091E80080FD1CC07C
:101D50008091F901882391F0853091F08091EB001A
:101D600085FD10C04091E4005091E50042175307F3
:101D700029F39A01915011F784E0089582E00895C3
:101D800083E0089581E0089580E008954091E8009F
:101D900042FFDECF08950E94390F0E94410FE0EE0E
:101DA000F0E0808181608083E8EDF0E080818F77D2
:101DB000808319BCA7EDB0E08C918E7F8C938081DD
:101DC0008F7E80831092F80108950F931F93CF9315
:101DD000DF930E94390F0E94410FC8EDD0E0888147
:101DE0008F77888388818068888388818F7D8883C6
:101DF00019BC1092F9011092F5011092F70110929E
:101E0000F60100EE10E0F80180818B7F80838881ED
:101E10008160888342E060E080E00E94450EE1EE50
:101E2000F0E080818E7F8083E2EEF0E0808181604F
:101E30008083808188608083F80180818E7F8083A9
:101E4000888180618883DF91CF911F910F910895E0
:101E5000E8EDF0E080818F7E8083E7EDF0E0808127
:101E60008160808384E082BF81E08093F8010C94DC
:101E7000E50EE8EDF0E080818E7F80831092E20035
:101E800008951092DA001092E10008951F920F92C7
:101E90000FB60F9211242F933F934F935F936F933D
:101EA0007F938F939F93AF93BF93EF93FF93809113
:101EB000E10082FF0BC08091E20082FF07C08091A9
:101EC000E1008B7F8093E1000E94AD118091DA00E8
:101ED00080FF1FC08091D80080FF1BC08091DA0076
:101EE0008E7F8093DA008091D90080FF0DC080E161
:101EF00089BD82E189BD09B400FEFDCF81E08093F8
:101F0000F9010E94A80B05C019BC1092F9010E94AA
:101F1000B60B8091E10080FF19C08091E20080FF44
:101F200015C08091E2008E7F8093E2008091E200F4
:101F300080618093E2008091D80080628093D80015
:101F400019BC85E08093F9010E94BA0B8091E100F1
:101F500084FF30C08091E20084FF2CC080E189BD05
:101F600082E189BD09B400FEFDCF8091D8008F7D4C
:101F70008093D8008091E1008F7E8093E100809172
:101F8000E2008F7E8093E2008091E2008160809386
:101F9000E2008091F501882311F084E007C0809170
:101FA000E30087FD02C081E001C083E08093F90176
:101FB0000E94BC0B8091E10083FF29C08091E20068
:101FC00083FF25C08091E100877F8093E10082E05C
:101FD0008093F9011092F5018091E1008E7F80934A
:101FE000E1008091E2008E7F8093E2008091E20028
:101FF00080618093E20042E060E080E00E94450E54
:102000008091F00088608093F0000E94B90BFF91EE
:10201000EF91BF91AF919F918F917F916F915F9160
:102020004F913F912F910F900FBE0F901F901895D9
:102030001F920F920FB60F9211242F933F934F933D
:102040005F936F937F938F939F93AF93BF93CF9340
:10205000DF93EF93FF93C091E900CF708091EC0084
:10206000D82FD17080FDD0E81092E9008091F00067
:10207000877F8093F00078940E945C101092E900B2
:102080008091F00088608093F000CD2BCF70C093DA
:10209000E900FF91EF91DF91CF91BF91AF919F91B7
:1020A0008F917F916F915F914F913F912F910F9001
:1020B0000FBE0F901F9018951F93CF93DF93CDB74E
:1020C000DEB7AA970FB6F894DEBF0FBECDBFEAEF1A
:1020D000F1E088E08E0F9091F10091938E13FBCF89
:1020E0000E94D80B8091E80083FF1FC18091FA0104
:1020F0009091FB01492F50E04A30510508F015C17D
:10210000FA01EC59FF4F0C944725803881F0823852
:1021100009F00BC18091FE018F708093E9008091DE
:10212000EB0085FB882780F91092E90006C08091BA
:10213000F6019091F701911182609091E800977FEC
:102140009093E8008093F1001092F100C8C0282F0E
:102150002D7F09F0EAC0882319F0823061F0E5C0D4
:102160008091FC01813009F0E0C0933009F080E0FB
:102170008093F7012BC08091FC01811127C08091D1
:10218000FE018F7009F4D1C08093E9002091EB002B
:1021900020FF1CC0933021F48091EB00806214C0BA
:1021A0009091EB0090619093EB0021E030E0A90169
:1021B00002C0440F551F8A95E2F74093EA0010923F
:1021C000EA008091EB0088608093EB001092E900B8
:1021D0008091E800877F86C08111A7C01091FC0123
:1021E0001F778091E3008078812B8093E3008091BA
:1021F000E800877F8093E8000E947A0E8091E800D3
:1022000080FFFCCF8091E30080688093E300111190
:1022100002C082E001C083E08093F90186C080584B
:10222000823008F082C08091FC019091FD018C3DCC
:1022300053E0950779F583E08A838AE289834FB773
:10224000F894DE01139620E03EE051E2E32FF0E047
:1022500050935700E49120FF03C0E295EF703F5F79
:10226000EF708E2F90E0EA3010F0C79601C0C09654
:102270008D939D932F5F243149F74FBF8091E800E4
:10228000877F8093E8006AE270E0CE0101960E94A9
:10229000810D14C0AE014F5F5F4F6091FE010E943F
:1022A000C80CBC01009709F440C09091E800977FEA
:1022B0009093E80089819A810E94E40D8091E80062
:1022C0008B778093E80031C0803879F58091E80001
:1022D000877F8093E8008091F5018093F1008091E1
:1022E000E8008E778093E8000E947A0E1EC081116C
:1022F0001CC09091FC019230C0F48091E800877F6F
:102300008093E8009093F5010E947A0E8091F50188
:10231000811106C08091E30087FD02C081E001C009
:1023200084E08093F9010E94C40B8091E80083FF50
:102330000AC08091E800877F8093E8008091EB00DD
:1023400080628093EB00AA960FB6F894DEBF0FBEB2
:10235000CDBFDF91CF911F9108950895CF938091C4
:10236000F9018823A1F0C091E900CF709091EC00B1
:10237000892F817090FD80E8C82B1092E900809130
:10238000E80083FD0E945C10CF70C093E900CF91FC
:10239000089590937D0180937C010895E0917C01E4
:1023A000F0917D01309721F00190F081E02D0994AA
:1023B00080E00895E0917C01F0917D01309721F05B
:1023C0000280F381E02D09940895E0917C01F09161
:1023D0007D01309721F00480F581E02D0994089566
:1023E00020917A0130917B018217930771F09093CD
:1023F0007B0180937A01E0917C01F0917D0130971F
:1024000021F00680F781E02D09940895209178014C
:10241000309179018217930771F09093790180933D
:102420007801E0917C01F0917D01309721F00084EA
:10243000F185E02D0994089508950C941C120E94D2
:10244000261D0E94A5030C94E81D9F92AF92BF9297
:10245000CF92DF92EF92FF920F931F93CF93DF9370
:1024600000D000D000D0CDB7DEB70E94BD030DE094
:1024700010E0AA24A394B12C902E802F0E94AB04CC
:10248000980121583E4F6901F901F080F826A1F426
:102490000150110988F78FEF89838A831B820E947C
:1024A0002F1D8160782F9D838C8349815A816B8198
:1024B0008D810E94BC122FC09091E20191FF04C057
:1024C0008E830E94B1048E8125E030E0A501022EAA
:1024D00001C0440F0A94EAF7E42E4F21C1F029838A
:1024E0009A828E2191E009F490E09B830E942F1D37
:1024F0008160782F9D838C8349815A816B818D8186
:102500000E94BC12F6018081E826E08204C02150BE
:102510003109E0F6BDCF0E94CF2010917E010E94CC
:10252000CE111817B9F00E94CE1180937E01269625
:102530000FB6F894DEBF0FBECDBFDF91CF911F91D4
:102540000F91FF90EF90DF90CF90BF90AF909F9052
:102550000C94C70A26960FB6F894DEBF0FBECDBF07
:10256000DF91CF911F910F91FF90EF90DF90CF906F
:10257000BF90AF909F900895CF93DF93CDB7DEB714
:102580002B970FB6F894DEBF0FBECDBF4F83588791
:1025900069877A878B87DE01119686E0FD011192AB
:1025A0008A95E9F785E0FE01379601900D928A95AC
:1025B000E1F749815A816B817C818D819E810E94E6
:1025C00005192B960FB6F894DEBF0FBECDBFDF9175
:1025D000CF910895CF93882309F4C2C0C82F8238C1
:1025E00059F40E94CE1181FDBBC089E30E94DF1B1C
:1025F0000E94AC1C89E30CC0833879F40E94CE1190
:1026000080FDAEC083E50E94DF1B0E94AC1C83E509
:102610000E94211CCF910C94AC1C843859F40E9468
:10262000CE1182FD9DC087E40E94DF1B0E94AC1C7E
:1026300087E4EECF8CEF8C0F813A48F48C2F0E9408
:10264000122381118DC08C2F0E94DF1BE3CF80E20B
:102650008C0F883048F4C77081E001C0880FCA959C
:10266000EAF70E94651CD6CF8BE58C0F833078F497
:10267000C53A29F0C63A31F083E890E005C081E818
:1026800090E002C082E890E0CF910C94F01188E5D0
:102690008C0F833108F064C0C83A39F1C93A41F16E
:1026A000CA3A49F1CB3A51F1CC3A59F1CD3A61F1FC
:1026B000C03B69F1CE3A71F1CF3A79F1C13B81F17A
:1026C000C23B89F1C33B91F1C43B99F1C53BA1F1F8
:1026D000C63BA9F1C73BB1F1C83BB9F1C93BC1F158
:1026E000CA3BC9F180E090E038C082EE90E035C08E
:1026F00089EE90E032C08AEE90E02FC085EB90E04A
:102700002CC086EB90E029C087EB90E026C08CECD3
:1027100090E023C08DEC90E020C083E891E01DC0E4
:102720008AE891E01AC082E991E017C084E991E05B
:1027300014C081E292E011C083E292E00EC084E214
:1027400092E00BC085E292E008C086E292E005C00C
:1027500087E292E002C08AE292E0CF910C940612E6
:10276000CF910895882309F44BC0823859F40E9410
:10277000CE1181FF45C089E30E94DF1B0E94AC1C83
:1027800089E30CC0833871F40E94CE1180FF38C0F9
:1027900083E50E94DF1B0E94AC1C83E50E94211C84
:1027A0000C94AC1C843859F40E94CE1182FF28C0CE
:1027B00087E40E94DF1B0E94AC1C87E4EFCF9CEFF4
:1027C000980F913A58F390E2980F983050F4877030
:1027D00091E001C0990F8A95EAF7892F0E946B1C3E
:1027E000DFCF9BE5980F933020F480E090E00C94CD
:1027F000F011885A833120F480E090E00C940612A6
:102800000895882321F00E94651C0C94AC1C089547
:10281000882321F00E946B1C0C94AC1C08957F92BD
:102820008F929F92AF92BF92CF92DF92EF92FF92E0
:102830000F931F93CF93DF931F92CDB7DEB77C0129
:10284000C62E772EFC01058102950F7012811111A1
:102850000E94821C0E94D81B882379F0112369F002
:1028600080E28C0D883048F082E00E94C11B0E94FB
:10287000D81B91E0D82ED92601C0D12CE72DE295A6
:10288000EF70F0E0E259FF4F0C944725872D807FD1
:10289000072D0F70882311F00295007F112389F016
:1028A000002309F490C180E28C0D883020F4802F41
:1028B0000E94651C03C0802F0E94751C0E94AC1CE6
:1028C00082C18C2D0E94B213002309F495C180E2CD
:1028D0008C0D883020F4802F0E946B1C03C0802F49
:1028E0000E947B1C0E94AC1C87C1972D907F872D76
:1028F0008F70903211F08295807FCC2021F0F1E032
:10290000CF16B1F01EC0112349F0002309F414C101
:10291000013009F011C10E94951C6EC1002319F00D
:10292000013009F469C189830E94981C89810AC118
:10293000112321F0023008F05FC1FEC001115CC11B
:1029400001C1112321F0002309F4F6C03CC100238A
:1029500009F4F8C03EC1872D86958695837090E076
:10296000009719F0019761F047C1112321F08C2DD8
:10297000972D937002C080E090E00E94F0113CC15E
:10298000112321F08C2D972D937002C080E090E0F0
:102990000E94061231C18C2D112319F00E94D71FFD
:1029A00002C00E943F200E94C42026C1872D837050
:1029B00009F052C0111120C18C2D82958695877027
:1029C000880F880F9C2D9F70892E912CA12CB12CE3
:1029D000082E04C0880C991CAA1CBB1C0A94D2F7B0
:1029E000C4FE14C00FE010E020E030E0B901A801FF
:1029F00004C0440F551F661F771F8A95D2F7CB017D
:102A0000BA01609570958095909503C060E070E084
:102A1000CB01272D26952695237030E022303105F5
:102A200069F02330310589F0682979298A299B29A1
:102A30002130310571F00E944D1ADEC068297929D4
:102A40008A299B290E94691AD7C00E944D1AC50184
:102A5000B4010E94311AD0C0112319F0872D817062
:102A600001C08695882309F4C7C08C2D8295869570
:102A70008770880F880F9C2D9F70892E912CA12C18
:102A8000B12C082E04C0880C991CAA1CBB1C0A94EB
:102A9000D2F7C4FE14C00FE010E020E030E0B9012E
:102AA000A80104C0440F551F661F771F8A95D2F7EF
:102AB000CB01BA01609570958095909503C060E058
:102AC00070E0CB01272D269526952370422F50E0EC
:102AD0004230510569F04330510589F06829792960
:102AE0008A299B294130510571F00E94271B84C01F
:102AF000682979298A299B290E94431B7DC00E944D
:102B0000271BC501B4010E940B1B76C08C2D90E0E1
:102B1000FC01E05EF109E531F10508F050C0E25832
:102B2000FF4F0C9447250C2D0F70872D8F711123AB
:102B300031F00E94A41A802F0E9401145DC00E94EF
:102B4000C51A802F0E94081457C0112339F00111B3
:102B500053C0872D8F710E94EA1A4EC0023008F0D0
:102B60004BC0F7CF112339F0872D8F710E94A41A23
:102B700043C01123C9F3872D8F710E94C51A3CC031
:102B8000112329F0872D8F710E948F1A35C00E9462
:102B9000851A32C0112351F0172D1F71812F0E9409
:102BA000A41A63E0812F0E94B81B26C081E00E9416
:102BB000C11B023008F182E00E94C11B1DC011231D
:102BC00031F0002389F28C2D0E94EA1215C00023F7
:102BD00091F28C2D0E94B2130FC0472D4F706C2DB7
:102BE000C7010E9487050E94A91906C0472D4F7092
:102BF0006C2DC7010E94D607DD20F9F00E94B41B9E
:102C000080FD1BC0F70112820E94AE1B0E94A41A15
:102C1000C7010E942C160E94AE1B0F90DF91CF912E
:102C20001F910F91FF90EF90DF90CF90BF90AF90EA
:102C30009F908F907F900C94C51A0F90DF91CF9149
:102C40001F910F91FF90EF90DF90CF90BF90AF90CA
:102C50009F908F907F9008950F931F93CF93DF9352
:102C6000EC01888199812B813C81232BB9F09F3F16
:102C700011F48F3F99F0CE010E942E07882371F046
:102C8000688179818A810E94AA1B8C010E945F1B46
:102C90000E94261AB801CE010E940F14DF91CF9135
:102CA0001F910F9108950E94821C0E94921C0E9405
:102CB000571C0E94AC1C0E9475210E94C42080E019
:102CC00090E00E94F01180E090E00C9406120E94C7
:102CD000721C0C9453160E949F1B292F22952F7053
:102CE00030E02C3031054CF42A3031056CF42250A0
:102CF000310922303105A8F407C02C30310569F0C4
:102D00002F30310551F00DC0803F69F018F4803E3E
:102D100040F409C0843F29F406C093FB882780F95A
:102D2000089580E0089581E00895CF93DF9300D067
:102D300000D01F92CDB7DEB70F900F900F900F907D
:102D40000F90DF91CF910895CF93DF9300D000D003
:102D500000D0CDB7DEB726960FB6F894DEBF0FBE13
:102D6000CDBFDF91CF9108951F93CF93DF93C09193
:102D70008D0116E080918E01C81799F0D0E01C9F5C
:102D8000F0011D9FF00D1124E157FE4F408151814C
:102D900062817381848195810E94A4162196C770F7
:102DA000E9CFDF91CF911F9108954091BF015091DC
:102DB000C0016091C1017091C2018091C3019091E5
:102DC000C4010C94A4168091C40182958F7009F0FF
:102DD00054C08091C101882309F44FC080918D01B6
:102DE000A0918E016091BF017091C0014091C2011C
:102DF0005091C301B6E08A1709F43FC090E0411535
:102E00005105C1F17F3F11F46F3FA1F1B89FF0016F
:102E1000B99FF00D1124E157FE4F218172132AC092
:102E20002081621327C02281211124C02381348193
:102E30002417350710F421503109241B350B283C89
:102E40003105C0F42091C4012F7020612093C4018A
:102E500026E0289FF001299FF00D1124EC56FE4F2B
:102E600080818F70806180838FEB91E00E942C16AF
:102E70000C94B41601968770BECF0895CF92DF925E
:102E8000EF92FF920F931F93CF93DF93CDB7DEB7EF
:102E900062970FB6F894DEBF0FBECDBF8C0185E000
:102EA000F801DE011D9601900D928A95E1F7D80197
:102EB0004C9111965C91119712966C911297139602
:102EC000CD90DC9014973091BF017091C00180913A
:102ED000C2019091C301009709F46BC17F3F19F4BF
:102EE0003F3F09F466C1E090C101EE2009F4C0C083
:102EF0002091C401C816D90628F0F601E81BF90B89
:102F0000CF0104C0809590958C0D9D1DFF24F394F6
:102F1000883C910578F0F12C207F09F0C6C07C2D0B
:102F2000D98AC88A89890E9495168FEB91E00E9400
:102F30002C16B1C0822F807F09F046C0751314C0D3
:102F4000341312C0611110C02F7020612093C4018E
:102F50000E94D5168FEB91E00E942C168091C4013F
:102F6000D80115968C932EC0CD2819F15F3F11F42E
:102F70004F3FF9F0F62E61111CC080918D01209118
:102F80008E0136E0821709F45AC090E0389FF001B4
:102F9000399FF00D1124E157FE4F7181571306C080
:102FA0007081471303C07281711103C0019687704D
:102FB000E9CFF62E662309F418C18091C40181601F
:102FC0008093C401F12C11C1751308C0341306C0DD
:102FD000611104C08091C401D801C3C04D875E87D0
:102FE0008D859E856A8B0E946B166A898823E1F124
:102FF0006623D1F12091C401822F82958F7090E0D9
:10300000029774F08091BF019091C00198878F83DF
:103010001986DB86CA862C87CE0107960E942C165D
:1030200086E0F801AFEBB1E001900D928A95E1F7EF
:103030000E94E3160E94D516FF24F394D6C04D8754
:103040005E878D859E850E949F1B292F22952F705C
:1030500030E0223031050CF0BCC09F7009F0B6C0E2
:10306000805E883008F4C1C0C8010E942C16E4CFED
:10307000C816D90608F453C0F601E81BF90BCF01B6
:10308000883C910508F450C0F12C7C2DD98AC88A5F
:1030900089890E949516EFEBF1E086E0DF011D9231
:1030A0008A95E9F70E94D516A0C0751314C0341391
:1030B00012C0611110C08091C401F8018583C8015C
:1030C0000E942C1686E0EFEBF1E0DF011D928A955D
:1030D000E9F7FE2C8AC04D875E878D859E856A8BB9
:1030E0000E946B166A89882309F4BECF662309F40F
:1030F000BBCF2091C401822F82958F7090E0029700
:103100000CF48ECF8091BF019091C0019A83898386
:103110001B82DD82CC822E83CE0101967FCF8095EB
:1031200090958C0D9D1DACCFF62E662309F49CCF97
:1031300075132EC034132CC02091C40120FD1FC074
:10314000822F82958F70D9F0D80115962C93159700
:103150008F3049F08F5F982F9295907F822F8F70DC
:10316000892B15968C93C8010E942C1686E0F801D5
:10317000AFEBB1E001900D928A95E1F793CF86E035
:10318000F801AFEBB1E001900D928A95E1F72DC007
:103190004D875E878D859E850E946B16811140CF7D
:1031A0008091C40181608093C401C8010E942C16E3
:1031B0001CC0662309F458CF4D875E878D859E8598
:1031C0000E946B16882309F44FCF2ACF811148CF74
:1031D0000CC0243031050CF047CF9F7009F440CF6C
:1031E000F8019581907F09F03BCF8F2D62960FB645
:1031F000F894DEBF0FBECDBFDF91CF911F910F912D
:10320000FF90EF90DF90CF9008951F93CF93DF93BF
:10321000CDB7DEB72C970FB6F894DEBF0FBECDBF8B
:103220004F83588769877A878B879C87CE0107965B
:103230000E943E17882369F08F8198852A853B85F7
:10324000232BF1F19F3F09F063C08F3F09F060C06D
:1032500037C086E0FE013796DE01119601900D928F
:103260008A95E1F76F817885EA85FB85309741F192
:103270007F3F11F46F3F21F120918E0130E0C901B1
:1032800001968770992740918D0150E0841795072A
:1032900009F447C069837A83FD83EC8396E0929FAB
:1032A000D001939FB00D1124A157BE4FFE0131965E
:1032B00001900D929A95E1F780938E010E94B416C9
:1032C00016E080918D0190918E018917C1F1189FB0
:1032D000C001112481579E4F0E943E17882379F127
:1032E000E0918D011E9FF0011124E157FE4F4081B6
:1032F000518162817381848195810E94A41680919D
:103300008D0190E001968770992780938D01D9CF28
:103310004F81588569857A858B859C850E94A41686
:10332000CFCF0E94671610928E0110928D01EFEBA5
:10333000F1E086E0DF011D928A95E9F7C1CF2C9676
:103340000FB6F894DEBF0FBECDBFDF91CF911F91B6
:103350000895EF92FF920F931F93CF93DF938C0109
:10336000009709F46CC0F12CEE24E394E801219657
:10337000F8018491843740F4843008F051C08130E2
:1033800081F0823019F15BC0853709F444C0A8F19F
:103390009CE7980F903708F052C08F770E94B213C5
:1033A00041C00E5F1F4FFE01C49180E28C0F883038
:1033B00048F4C7708E2D01C0880FCA95EAF70E94A5
:1033C000851C14C08C2F0E94EA122DC00E5F1F4F67
:1033D000FE01C49180E28C0F883058F4C7708E2DA6
:1033E00001C0880FCA95EAF70E948B1C0E94AC1C92
:1033F0001AC08C2F0E94B21316C00E5F1F4FFE0121
:10340000C491CC2381F08FE99FE00197F1F700C0D0
:103410000000C150F6CF0E5F1F4FFE01F49003C0B5
:103420000E94EA128E018F2D882309F49FCFEFE9C5
:10343000FFE03197F1F700C000008150F5CFDF9138
:10344000CF911F910F91FF90EF9008950895609391
:10345000C9017093CA018093CB019093CC010C9465
:1034600053160F931F930091C9011091CA01209127
:10347000CB013091CC01DC01CB01802B912BA22B15
:10348000B32B8093C9019093CA01A093CB01B09351
:10349000CC011F910F910C9453160F931F93009121
:1034A000C9011091CA012091CB013091CC01DC01FE
:1034B000CB0180239123A223B3238093C90190934E
:1034C000CA01A093CB01B093CC011F910F910C9432
:1034D00053160F931F930091C9011091CA012091B7
:1034E000CB013091CC01DC01CB0180279127A227B1
:1034F000B3278093C9019093CA01A093CB01B093E5
:10350000CC011F910F910C9453161092C50110928B
:10351000C6011092C7011092C8010C94531641E0E5
:1035200050E060E070E004C0440F551F661F771F35
:103530008A95D2F74093C5015093C6016093C701A5
:103540007093C8010C94531641E050E060E070E0C5
:1035500004C0440F551F661F771F8A95D2F78091CC
:10356000C5019091C601A091C701B091C801482B37
:10357000592B6A2B7B2B4093C5015093C601609356
:10358000C7017093C8010C94531641E050E060E00D
:1035900070E004C0440F551F661F771F8A95D2F74D
:1035A00040955095609570958091C5019091C601A8
:1035B000A091C701B091C801482359236A237B23F6
:1035C0004093C5015093C6016093C7017093C80131
:1035D0000C94531641E050E060E070E004C0440FEA
:1035E000551F661F771F8A95D2F78091C50190916C
:1035F000C601A091C701B091C801482759276A2781
:103600007B274093C5015093C6016093C701709317
:10361000C8010C9453160F931F930091C50110918C
:10362000C6012091C7013091C801DC01CB01802B7C
:10363000912BA22BB32B8093C5019093C601A0932D
:10364000C701B093C8011F910F910C9453160F93AB
:103650001F930091C5011091C6012091C7013091BF
:10366000C801DC01CB0180239123A223B3238093E3
:10367000C5019093C601A093C701B093C8011F91E3
:103680000F910C9453160F931F930091C501109145
:10369000C6012091C7013091C801DC01CB01802710
:1036A0009127A227B3278093C5019093C601A093C9
:1036B000C701B093C8011F910F910C945316089540
:1036C000CF92DF92EF92FF920F931F93CF93DF93EE
:1036D0008C01C090C901D090CA01E090CB01F0905C
:1036E000CC018091C5019091C601A091C701B09114
:1036F000C801C82AD92AEA2AFB2ACFE1D0E0D7019B
:10370000C6010C2E04C0B695A795979587950A9487
:10371000D2F780FF06C0B8018C2F0E942C0A0197B7
:1037200021F4219760F780E001C08C2FDF91CF91C9
:103730001F910F91FF90EF90DF90CF900895CF935E
:10374000DF93EC010E94601BBE010E942C0ADF91F6
:10375000CF910895CB010E949F1B08958091CD01C8
:1037600085958595859508958091CD0187700895FB
:1037700098E0899F90011124262B2093CD010C9471
:10378000A41A2091CD01809582238093CD01982F9A
:10379000977069F430E0482F552747FD509524175E
:1037A000350729F08595859585950C94C51A08955A
:1037B0009091CD01977081E009F480E00895909197
:1037C0000C01992321F090910D01911109C02091D4
:1037D0000E0130910F01F90132969FEF40E01FC0BA
:1037E000982F9695969596959F3050F5E0910E01FD
:1037F000F0910F01E90FF11D877021E030E0A90180
:1038000002C0440F551F8A95E2F7CA019181892BA6
:10381000818308959F3F39F04F5F4E3041F05191C1
:103820005813F8CF0DC05111F7CF942FF5CF9F3F0C
:1038300039F0F901E90FF11D97FDFA95828308959A
:10384000089590910C01992321F090910D0191110F
:1038500009C020910E0130910F01F9013296205FCD
:103860003F4F1FC0982F9695969596959F30F0F4F0
:10387000E0910E01F0910F01E90FF11D877021E039
:1038800030E0A90102C0440F551F8A95E2F7CA0132
:10389000809591818923818308953196E217F307FA
:1038A00029F090819813F9CF1082F7CF089581E025
:1038B00090E0E0910E01F0910F01E80FF91F1082E6
:1038C000019680319105A9F708959091E101892B26
:1038D0008093E101089580959091E101892380937F
:1038E000E10108951092E10108959091E001892B82
:1038F0008093E001089580959091E0018923809361
:10390000E00108951092E00108959091DF01892B64
:103910008093DF01089580959091DF018923809342
:10392000DF0108951092DF0108958093CE0108957C
:103930001092CE01089580910E0190910F01FC012B
:1039400031969C01205F3F4F80E0919191118F5FF4
:10395000E217F307D1F70895E0910E01F0910F01FE
:103960008091E1018083E0910E01F0910F0190813F
:103970008091E001892B8083E0910E01F0910F018D
:1039800090818091DF01892B80838091CE018823F3
:1039900061F0E0910E01F0910F019081892B8083FD
:1039A0000E949B1C81111092CE0180910E0190917A
:1039B0000F010C94DA1120E0009739F0AC0141506E
:1039C0005109842395232F5FF7CF822F089580918B
:1039D000F901843021F11092E30120E488E190E0C4
:1039E0000FB6F894A895809360000FBE20936000F6
:1039F00080E00E94C70A83B7817F846083BF83B75A
:103A0000816083BF7894889583B78E7F83BF88E178
:103A10000FB6F89480936000109260000FBE089576
:103A2000089508950E94101D0E94BD030E94111D5B
:103A30000E94B20491E0811101C090E0892F0895A5
:103A40000E9467160E94CE110C94C70A82E084BDC2
:103A500093E095BD9AEF97BD80936E0008952FB7C0
:103A6000F8948091E4019091E501A091E601B09174
:103A7000E7012FBF0895CF92DF92EF92FF920F934D
:103A80001F932FB7F8944091E4015091E5016091A4
:103A9000E6017091E7012FBF6A017B01EE24FF244C
:103AA0008C0120E030E0C016D106E206F30610F4E7
:103AB000415051099A01281B390BC9011F910F91DF
:103AC000FF90EF90DF90CF9008951F920F920FB666
:103AD0000F9211248F939F93AF93BF938091E40132
:103AE0009091E501A091E601B091E7010196A11D39
:103AF000B11D8093E4019093E501A093E601B0939A
:103B0000E701BF91AF919F918F910F900FBE0F90E2
:103B10001F9018950E94CB0EF8942FEF87EA91E63C
:103B2000215080409040E1F700C0000087E090EB1A
:103B3000DC018093030290930402A0930502B093EA
:103B400006029CE088E10FB6F894A8958093600087
:103B50000FBE90936000FFCFEF92FF920F931F93E1
:103B6000CF93DF93D82FCDE08C2F0E94AB0405E0DC
:103B700010E0E82EF12CC701002E02C09595879524
:103B80000A94E2F780FF09C0602F7C2F80E00E943A
:103B9000D707D81302C081E006C00150110958F7B9
:103BA000C15010F780E0DF91CF911F910F91FF90EE
:103BB000EF900895CF93C82F8CE20E94AC1D88230C
:103BC00021F08C2FCF910C94AC1D80E0CF91089503
:103BD000CF930E942F1F811102C00E94151FC5E6BE
:103BE000C15049F00E94BD038FE39CE90197F1F7B2
:103BF00000C00000F5CF89E20E94DA1D811113C1D7
:103C00008AE20E94DA1D81110E94151F85E00E9440
:103C1000DA1D81110E948A1D0E943A1F8093E201E1
:103C200087E00E94DA1D8823A9F18BE10E94DA1D4A
:103C3000882351F08091E20181FB222720F991E055
:103C4000922790FB81F90EC08EE00E94DA1D882336
:103C500061F08091E20182FB222720F991E0922716
:103C600090FB82F98093E20115C080E10E94DA1D89
:103C70009091E201882341F093FB222720F981E013
:103C8000822780FB93F904C0892F809580FB90F9EF
:103C90009093E2018091E2010E943E1F0E944C1F1E
:103CA0008093020280EE0E94DA1D882341F0809109
:103CB0000202982F909590FB80F98093020289E38D
:103CC0000E94DA1D882359F08091020281FB22278D
:103CD00020F991E0922790FB81F98093020282EE15
:103CE0000E94DA1D882359F08091020282FB22276C
:103CF00020F991E0922790FB82F98093020286EEF0
:103D00000E94DA1D882359F08091020283FB22274A
:103D100020F991E0922790FB83F98093020283EED1
:103D20000E94DA1D882359F08091020284FB222729
:103D300020F991E0922790FB84F98093020285E3B9
:103D40000E94DA1D882359F08091020285FB222708
:103D500020F991E0922790FB85F98093020281E39C
:103D60000E94DA1D882359F08091020286FB2227E7
:103D700020F991E0922790FB86F98093020281E17D
:103D80000E94DA1D882359F08091020287FB2227C6
:103D900020F991E0922790FB87F9809302028091AD
:103DA00002020E94501F8091020287FB882780F93F
:103DB00080930D0187E20E94DA1DC82F8EE10E94D8
:103DC000DA1D8111C2608FE10E94DA1D8111C46089
:103DD00080E20E94DA1D8111C86081E20E94DA1D32
:103DE0008111C06182E20E94DA1D8111C06283E20A
:103DF0000E94DA1D8111C06484E20E94DA1D8823CA
:103E000011F0C06802C0CC2329F08C2F0E94471FFC
:103E10006C2F03C00E94431F682F70E080E090E089
:103E2000CF910C94271ACF9108956DEE7EEF80E02C
:103E300090E00E94812560E082E090E00E946F2582
:103E400060E083E090E00E946F2560E084E090E015
:103E50000E946F2560E085E090E00C946F2580E083
:103E600090E00E94692521E08D3E9E4F09F020E000
:103E7000822F089582E090E00C946125682F82E003
:103E800090E00C946F2583E090E00C946125682FFE
:103E900083E090E00C946F2584E090E00C94612521
:103EA000682F84E090E00C946F258091EA0180FFF8
:103EB0000BC06091130185E0689FB00111247595D6
:103EC0006795759567952BC081FF09C060911301B7
:103ED00085E0689FB00111247595679520C082FF29
:103EE00007C06091130185E0689FB001112417C0DD
:103EF0009091EB019923D1F060911201961788F708
:103F00002091130185E0289F90011124929FA00128
:103F1000939F500D112470E0CA010E943325603830
:103F2000710540F46115710539F002C065E070E07B
:103F3000862F08958FE7089581E008958091EA0122
:103F400080FF08C06091110170E0759567957595C7
:103F5000679521C081FF06C06091110170E07595E1
:103F6000679519C082FF04C06091110170E010C014
:103F70009091EB019923C1F0609110019617A0F781
:103F800080911101899FC001112470E00E943325A6
:103F90006038710528F46115710521F0862F0895A8
:103FA0008FE7089581E0089561E070E0F4CF803FED
:103FB00021F40E94551F819504C0813F29F40E947D
:103FC000551F8093EE010895823F21F40E94551FF2
:103FD000819504C0833F29F40E94551F8093ED0111
:103FE0000895893F19F40E949E1F05C08A3F31F44D
:103FF0000E949E1F81958093EF0108958B3F21F4CD
:104000000E949E1F819504C08C3F29F40E949E1F30
:104010008093F0010895843F21F48091EC01816048
:1040200017C0853F21F48091EC01826011C0863F6A
:1040300021F48091EC0184600BC0873F21F48091D2
:10404000EC01886005C0883F31F48091EC0180610B
:104050008093EC0108958D3F21F48091EA01816005
:104060000BC08E3F21F48091EA01826005C08F3F32
:1040700029F48091EA0184608093EA010895803FE9
:1040800039F48091EE0187FF6CC01092EE0169C097
:10409000813F29F48091EE011816BCF362C0909123
:1040A000ED01823F29F497FF5CC01092ED0159C0E9
:1040B000833F19F41916CCF354C0893F41F4809121
:1040C000EF0118160CF04DC01092EF014AC08A3F64
:1040D00029F48091EF0187FF44C0F6CF8B3F39F47C
:1040E0008091F00187FF3DC01092F0013AC08C3FF3
:1040F00029F48091F0011816BCF333C0843F21F4F9
:104100008091EC018E7F17C0853F21F48091EC01F6
:104110008D7F11C0863F21F48091EC018B7F0BC015
:10412000873F21F48091EC01877F05C0883F31F4FF
:104130008091EC018F7E8093EC0113C08D3F21F4C0
:104140008091EA018E7F0BC08E3F21F48091EA01BD
:104150008D7F05C08F3F29F48091EA018B7F80938A
:10416000EA018091ED0181110EC08091EE01811173
:104170000AC08091EF01811106C08091F001811188
:1041800002C01092EB0108958CEE91E00E94E511BF
:104190000E942F1D9093E9018093E80108951F93D9
:1041A000CF93DF938091E8019091E9010E943B1D3C
:1041B000AC019091EB01992321F02091140130E0A2
:1041C00006C0209115018AE0289F90011124421712
:1041D000530708F486C08091ED01C091EE01D091A3
:1041E000EF011091F001811107C0C11176C0D1110A
:1041F00074C0111172C075C09F3F19F09F5F9093FA
:10420000EB01181624F40E94551F8093ED01809154
:10421000ED0187FF05C00E94551F81958093ED0138
:104220001C1624F40E94551F8093EE018091EE012C
:1042300087FF05C00E94551F81958093EE01609114
:10424000ED01662339F1C091EE01CC2319F17727F6
:1042500067FD7095872F972F0E94442423E333E353
:1042600043E35FE30E94A8240E9411246093ED01C0
:104270006C2F772767FD7095872F972F0E94442416
:1042800023E333E343E35FE30E94A8240E94112465
:104290006093EE011D1624F40E949E1F8093EF018F
:1042A0008091EF0187FF05C00E949E1F819580933A
:1042B000EF01111624F40E949E1F8093F00180915B
:1042C000F00187FF05C00E949E1F81958093F00139
:1042D000DF91CF911F910C94C4209F3F09F08ECFA6
:1042E00096CFDF91CF911F910895ECEEF1E085E03C
:1042F000DF011D928A95E9F71092EB011092EA0115
:104300000895833081F128F4813059F08230D1F062
:104310000895853009F449C0B8F1863009F456C0D3
:10432000089580911501262F30E0280F311D2F3F71
:10433000310524F4680F6093150108958FEF809381
:104340001501089580911401262F30E0280F311DAA
:104350002F3F310524F4680F6093140108958FEF07
:1043600080931401089580911301262F30E0280FC7
:10437000311D2F3F310524F4680F60931301089518
:104380008FEF80931301089580911201262F30E062
:10439000280F311D2F3F310524F4680F609312015F
:1043A00008958FEF80931201089580911101262FB7
:1043B00030E0280F311D2F3F310524F4680F609342
:1043C000110108958FEF80931101089580911001DC
:1043D000262F30E0280F311D2F3F310524F4680FC0
:1043E0006093100108958FEF80931001089583303A
:1043F00011F128F4813049F0823091F00895853030
:1044000081F120F18630C1F108958091150168177E
:1044100020F4861B809315010895109215010895CC
:1044200080911401681720F4861B8093140108956D
:1044300010921401089580911301681720F4861BCF
:104440008093130108951092130108958091120131
:10445000681720F4861B80931201089510921201B0
:10446000089580911101681720F4861B8093110133
:10447000089510921101089580911001681720F499
:10448000861B8093100108951092100108950F93D8
:104490001F938D3109F46BC008F03FC08E3009F4D2
:1044A0007FC0C0F4873009F469C068F4863009F031
:1044B000B1C08091E201817F8E7F8093E20181E033
:1044C0008093F201A8C0883009F4A2C08B3009F4AF
:1044D0009FC0A0C0863109F49BC078F4803109F4F4
:1044E00072C0813109F096C00E94671690910D014B
:1044F00081E0892780930D018BC0893109F488C040
:104500008B3109F087C08091E20181FB222720F9DD
:1045100091E0922790FB81F94CC0853309F470C07B
:1045200048F4873209F46CC008F459C0893209F4A0
:1045300067C070C0833438F48A3308F04EC08833C3
:1045400009F466C067C0833409F45AC0883409F09E
:1045500061C00E9467160FEF13ED20E30150104079
:104560002040E1F700C000000E948A1D51C00E9457
:10457000CB230E94CE110E94C70A4AC09091E2014B
:10458000892F8095817080FB90F929F09660986062
:104590009093E20140C0997F977F9093E20138C0E9
:1045A0008091E20182FB222720F991E0922790FB83
:1045B00082F98093E201992359F18091E2018160AF
:1045C0008093E20125C08091E20183FB222720F93C
:1045D00091E0922790FB83F9ECCF895301C08D5174
:1045E00041E050E060E070E08A019B0104C0000FF0
:1045F000111F221F331F8A95D2F7C901B80104C0C9
:1046000061E070E080E090E00E94271A0E94671647
:1046100081E001C080E01F910F91089580E008952E
:1046200080E00895CF93C82F8091F201813079F016
:1046300018F08230E9F187C0E0910E01F0910F018E
:104640008081813169F0823209F07FC009C0E09138
:104650000E01F0910F018081813111F0823261F4FD
:104660008C2F0E940E23811104C08C2F0E944722A0
:104670001DC081E090E01AC08C2F0E941023811190
:1046800014C0C43179F048F4CB3079F0C03109F06E
:1046900060C082E08093F20108C0C93219F0C833CB
:1046A00021F057C01092F20154C081E0817053C0D4
:1046B000C93289F118F5C43171F1A8F4C73009F095
:1046C00046C08AE08093150194E19093140193E031
:1046D000909313018093120188E08093110188E286
:1046E0008093100134C0CE51C63088F5EC2FF0E035
:1046F000E65DFE4F80818093F10129C0CE34E9F060
:1047000020F4CB3421F56AE013C0C13579F0C2350D
:10471000F1F461E00DC08091F101882319F010924D
:10472000F10115C081E08093F20115C061E006C07F
:104730008091F1010E9481210AC06AE08091F1011B
:104740000E94F72104C01092F20180E004C081E0D1
:1047500002C080E0ABCFCF910895E1E8F0E0808126
:10476000886080838081816080838FB7F89493E034
:104770009093890090ED909388008FBF0895EFE6A5
:10478000F0E08081826080830895EFE6F0E0808130
:104790008D7F80830895EFE6F0E0908182E08927A5
:1047A000808308951F920F920FB60F9211242F93BA
:1047B0003F934F935F936F937F938F939F93AF93A9
:1047C000BF93EF93FF938091F3019091F4010196D1
:1047D0009093F4018093F301811103C082E00E9461
:1047E000C70AE091F401E695E695F0E0E856FA4F45
:1047F000E4918091F3018E1303C080E00E94C70A08
:10480000FF91EF91BF91AF919F918F917F916F91A8
:104810005F914F913F912F910F900FBE0F901F907E
:10482000189504D06894B1118DC0089570D088F0A7
:104830009F5790F0B92F9927B751A0F0D1F0660F8C
:10484000771F881F991F1AF0BA95C9F712C0B130A7
:1048500081F077D0B1E0089574C0672F782F882752
:10486000B85F39F0B93FCCF3869577956795B395E6
:10487000D9F73EF490958095709561957F4F8F4F55
:104880009F4F0895E89409C097FB3EF4909580955A
:10489000709561957F4F8F4F9F4F9923A9F0F92F06
:1048A00096E9BB279395F695879577956795B79584
:1048B000F111F8CFFAF4BB0F11F460FF1BC06F5F6A
:1048C0007F4F8F4F9F4F16C0882311F096E911C07C
:1048D000772321F09EE8872F762F05C0662371F09D
:1048E00096E8862F70E060E02AF09A95660F771FB1
:1048F000881FDAF7880F9695879597F9089557FDE1
:104900009058440F551F59F05F3F71F04795880F3D
:1049100097FB991F61F09F3F79F0879508951216D4
:1049200013061406551FF2CF4695F1DF08C0161680
:1049300017061806991FF1CF869571056105089431
:104940000895E894BB2766277727CB0197F9089548
:104950000BD078C069D028F06ED018F0952309F0FC
:104960005AC05FC01124EECFCADFA0F3959FD1F3E8
:10497000950F50E0551F629FF001729FBB27F00D0D
:10498000B11D639FAA27F00DB11DAA1F649F662762
:10499000B00DA11D661F829F2227B00DA11D621FB1
:1049A000739FB00DA11D621F839FA00D611D221F6B
:1049B000749F3327A00D611D231F849F600D211D4F
:1049C000822F762F6A2F11249F5750408AF0E1F0F2
:1049D00088234AF0EE0FFF1FBB1F661F771F881F3B
:1049E00091505040A9F79E3F510570F014C0AACFD6
:1049F0005F3FECF3983EDCF3869577956795B79526
:104A0000F795E7959F5FC1F7FE2B880F911D96954F
:104A1000879597F9089597F99F6780E870E060E0BF
:104A200008959FEF80EC089500240A941616170647
:104A300018060906089500240A941216130614068F
:104A400005060895092E0394000C11F4882352F0F2
:104A5000BB0F40F4BF2B11F460FF04C06F5F7F4FAA
:104A60008F4F9F4F089597FB072E16F4009407D0A1
:104A700077FD09D00E944D2507FC05D03EF49095A6
:104A800081959F4F0895709561957F4F0895EE0F22
:104A9000FF1F0590F491E02D0994AA1BBB1B51E167
:104AA00007C0AA1FBB1FA617B70710F0A61BB70B9E
:104AB000881F991F5A95A9F780959095BC01CD0143
:104AC0000895F999FECF92BD81BDF89A992780B5D6
:104AD0000895A8E1B0E042E050E00C948925262F2B
:104AE000F999FECF92BD81BDF89A019700B40216E4
:104AF00039F01FBA20BD0FB6F894FA9AF99A0FBE92
:104B000008950196272F0E9470250C946F25DC01D3
:104B1000CB01FC01F999FECF06C0F2BDE1BDF89AC8
:104B2000319600B40D9241505040B8F70895F89472
:024B3000FFCFB5
:104B32000220C90A570B340B000BCC0A0101CF012A
:104B420028080A03140A3F4D363959050C05D604C4
:104B52009D043004490462047B0401020304050637
:044B62000708090037
:00000001FF
